:100000008A110A1205280000090007309F00831694
:100010008501E030860083120511851183160511D4
:100020008511F030860583126430A0000030A100F5
:10003000FC2233305A2333305A2333305A232230B0
:100040005A2328305A230C305A2301305A23B9013D
:10005000BA013810BB01BC01BD01BE01BF01C00126
:10006000B810C101C2013810BB01B810C101C201F2
:1000700005130530B6000130B70083160510831252
:100080000530B4000230B500831685108312AB230F
:10009000AB2301305A2380305A233330412335308B
:1000A0004123433041234D304123203041235430FC
:1000B00041235830412320304123553041234D30D6
:1000C000412341304123313041233030412331300D
:1000D000412334304123543041236430A000A10136
:1000E000FC22003083169B001C1400001A088312A7
:1000F000BC0038303C0203187E2884281F3083055A
:100100003C08443C0318A428003083169B00383078
:100110009A001C1555309D00AA309D009C149C1817
:100120008F281C1183128C13013083169B00003022
:100130009A001C1555309D00AA309D009C149C18F7
:100140009F281C1183128C131F30830500308316E7
:100150009B001C1400001A088312B900013083169A
:100160009B001C1400001A088312BA00D321282215
:10017000CB305A2320304123573041234130412393
:1001800049304123543041236430A000A101FC22B6
:100190000922CA283B08013C031DCF2883211F30B8
:1001A00083053B08023C031DDA281F308305861AAD
:1001B000DA2899211F3083053B08023C031DEC28F7
:1001C0001F308305861EEC284108013EC10042080D
:1001D0000318013E003EC2001F3083054108A00005
:1001E0004208A1004E30A3002030E022031D122956
:1001F0001F308305861E1229C101C20100308316FB
:100200009B001C1400001A088312B90001308316E9
:100210009B001C1400001A088312BA00BB01B8101E
:10022000D32109221F308305861F21291F30830512
:10023000061F21291F308305381821293814C101D0
:10024000C2011F308305381C2F291F308305861BF0
:100250002F291F308305061F2F29381048211F30F2
:100260008305381C3D291F308305861F3D291F301B
:100270008305061B3D29381068211F3083053B0884
:10028000003C031D442909221F308305CA28472941
:100290003A080A3EBA0064303A02031C5329BA01F4
:1002A0003908013EB9001F3083053908443C031D5D
:1002B00062291F3083053A08003C03186229443044
:1002C000B900BA011F3083050130BB00832108004B
:1002D0000A303A02BA003A08643C031874295A30CA
:1002E000BA0001303902B9001F30830538303902B5
:1002F00003187D293830B900BA011F308305013059
:10030000BB00832108003B08013C031D9629CB302C
:100310005A232030412354304123553041234E305D
:100320004123453041230230BB00D3211F308305D8
:100330000800BB01B8100513003083169B00831220
:10034000390883169A001C1555309D00AA309D006F
:100350009C149C18A9291C1183128C13013083163C
:100360009B0083123A0883169A001C1555309D0095
:10037000AA309D009C149C18BB291C1183128C135D
:100380002822CB305A23203041235730412341309B
:1003900041234930412354304123E830A000033049
:1003A000A100FC220800C0305A230A303A02031888
:1003B000F029383041233908A400A50170232E30DC
:1003C0004123303041233A08A400A5017023203096
:1003D00041234D304123483041237A304123062ABE
:1003E0001F308305383041233908A400A50170234C
:1003F0002E3041233A08A400A50170232030412368
:100400004D304123483041237A3041231F3083054A
:1004100008003B08003C031D252A1F308305B8183F
:10042000252A2822B830A0000B30A100FC22CB30B6
:100430005A234F3041234E3041234130412349302C
:100440004123523041230517B8141F30830508009B
:100450002030A0000330A1000030A2000030A30033
:100460003908A4000001A5000001A6000001A700B2
:10047000D5232008BD002108BE002208BF002308A4
:10048000C0003D08AC003E08AD003F08AE0040088B
:10049000AF001030A4002730A5000030A6000030C7
:1004A000A700FE232008BD002108BE002208BF00CF
:1004B0002308C0006430AC000030AD000030AE0056
:1004C0000030AF003A08A4000001A5000001A6001A
:1004D0000001A700FE232008C3002108C400220851
:1004E000C5002308C6003D08A0003E08A1003F0843
:1004F000A2004008A3004308A4004408A500450842
:10050000A6004608A700D5232008C3002108C40080
:100510002208C5002308C6004308BD004408BE00E9
:100520004508BF004608C0003D08A0003E08A100E5
:100530003F08A2004008A300FA30A4000030A50044
:100540000030A6000030A7002A242C08BD002D088A
:10055000BE002E08BF002F08C000A8230616C63014
:100560008F23F8308F2325308F23A4308F233E082C
:100570008F233D088F23AB230800BD2A1030A6002F
:10058000A501A401210DA40DA50D2208A402230894
:10059000031C230FA5020318D42A2208A40723084A
:1005A0000318230FA5070310A00DA10DA60BC22A47
:1005B00020080800A2000530EC2AA2000230EC2A34
:1005C000A2000630EC2AA2000330EC2AA20004307C
:1005D000EC2AA2000130EC2AA80023082102031D06
:1005E000F32A2208200204300318013003190230D4
:1005F0002805031DFF300800A0080319072B0E2350
:10060000A00300000000000000000000FC2AA10878
:10061000031908000E23A103A003FC2A0C30A50037
:10062000A50B102B000000001230A200A20B1D2B06
:100630001F231F230000000008001F23162B0D306E
:10064000A400A40B212B000008000A30A802031C00
:1006500008002A2B0630A802031C08002A2B1030A1
:10066000A8020001031C013EA902031C0800382B4C
:100670000A30A8020001031C013EA902031C080065
:10068000382BA8008515A80EF030860528080F39EC
:1006900086045523A80EF030860528080F398604F5
:1006A00055236430A8002523080005150000051116
:1006B00000000800A8008511A80EF0308605280863
:1006C0000F3986045523A80EF030860528080F3907
:1006D00086045523B830A8000B30A9002F2308004A
:1006E000A7172730A300103081230330A300E83080
:1006F0008123A30164308123A3010A3081232408CC
:100700008C2BA2002508A1002408A000BE222008EE
:10071000031DA713A71B0800303E41230800A000BB
:100720000830A100A00D0318AE23031CB323B82387
:10073000BD23A10B922BC923A023CF23B3230800F1
:10074000B8233608840037080005FF3EBD230800A3
:10075000B323BD23C62BB823AE23C62B3608840093
:1007600037088004C22B3608840037098005C22B65
:100770003408840035088004C22B3408840035090D
:100780008005C22B84170009841380050000000037
:1007900008003608840084173708800408003608EB
:1007A000840084173709800508002408A00703186F
:1007B000E4232508A1070318E7232608A207031846
:1007C000EA232708A3070800A10A031D0800A20ABC
:1007D000031D0800A30A0800EF23D5230800A4097D
:1007E000A509A609A709A40A031D0800A50A031D57
:1007F0000800A60A031D0800A70A0800A001A1011D
:10080000A201A3012C3084000430AA00082C242467
:100810000018D52324248018D52324240019D52397
:1008200024248019D5232424001AD5232424801AB3
:10083000D5232424001BD5232424801BD523840AFC
:10084000AA03031D072C08000310A40DA50DA60D77
:10085000A70D0800AC01AD01AE01AF01A71F312CFF
:100860000800EF23A71B352C0800AB01271F3B2CEA
:10087000AB0A2424362C2308B3002208B200210836
:10088000B1002008B000D523A31F4F2C3308A300CC
:100890003208A2003108A1003008A000702C2B08FB
:1008A000073C031C552C2C30622C2B080F3C031CDE
:1008B0005B2C2D30622C2B08173C031C612C2E3036
:1008C000622C2F3084002B080739AA000130A900C0
:1008D00003196E2C0310A90DAA0B6A2C2908800499
:1008E0000314A70CA60CA50CA40CAB03AB1F3B2C4C
:0208F0000800FE
:02400E00503F21
:0442000000001500A5
:00000001FF
